:030000000219FDE5
:03000B000200AA46
:03002B0002015976
:03005B000202EBB3
:030073000202D8AE
:1000800002030406080C10182030406080040608A3
:100090000C10182030406080A0C00003070F1F0D17
:1000A0000D04050D050205030302C2AFC0D0C0E078
:1000B000206214E5256009E473E525F4F58AD2622F
:1000C000D0E0D0D0D2AF3285268AC262E526F46075
:1000D0002AD0E0D0D0C295C294C293D2AF32C2959A
:1000E000C294C293206F0D20660A7405D5E0FDE529
:1000F0007BF45290D0E0D0D0D2AF32758A00C28D5E
:10010000D26201F401B9306805206602D29501B9C6
:10011000306805206602D29401B930680520660275
:10012000D29301B9D29230680A2066077403D5E0F1
:10013000FDD29501B9D29130680A2066077403D5C3
:10014000E0FDD29401B9D290D29230680A206607BD
:100150007403D5E0FDD29301B9C2AFC2AD53E6EF4F
:10016000C0D0C0E0D2D3D2AFC2CEE52A600720749F
:1001700049152A21BA7800790020742EE580307E56
:1001800001F430E70278FF53DACF207E0343DA2010
:10019000307E0343DA10C2D8C271E580307E01F4AC
:1001A00030E70279FFC3E89970CB306103752A18F4
:1001B000207403752A18885CD27020740DE52B60BA
:1001C00004152B21CA43DA01C2D82070024139A894
:1001D0005C206102C2702074367982B70431C3E8B2
:1001E00094F0400374F0F8E8C4540F28F87984B709
:1001F0000302410FC313C3138721200802C3132036
:100200000A06C3C898F8410F28F8500374FFF8880D
:1002100022E52D54066022206B1FE536C333C3331D
:10022000F8E564C313C313F9C3952240028922E899
:100230002522F52250037522FF7882B6044E8522CE
:1002400024A824C3E52495614002A861C3E895630E
:100250004002A8638825E5667002418AC3E8AA6661
:100260009A5003E8FAE4F9EAC333FBE568F45B2942
:10027000400D2567F8E56760021567400B418A0A63
:10028000C3E5679A5002056778FF8826C3E5259481
:10029000404002D26420CF0AD0E0D0D043E610D252
:1002A000AD32C2CF053A7801E52A600530740215F7
:1002B0002AC3E55C94014005755F0041CE7560007E
:1002C000756900E55F2401F55F5003755FFFD0E0BD
:1002D000D0D043E610D2AD32C2AF53E67F7592FA6A
:1002E0007593FFC260759104D2AF32C2AF53E6EF8F
:1002F000C2ADC0D0C0E0C0F0D2D3D2AFA8FBA9FC41
:10030000C2D8307102615253DACF207E0343DA1033
:10031000307E0343DA20D271E580307E01F420E79D
:1003200002612988278928A17F53DACF207E0343E1
:10033000DA20307E0343DA10C2D8C271307402A1D1
:100340006B7800E580307E01F430E702A16B885CB9
:10035000A15353DACF207E0343DA20307E0343DA01
:1003600010C271206102812B53DACF207E0343DA61
:1003700010307E0343DA20C2D8D27188578958C31F
:10038000E89555F8E99556F97B007E087A00C3E8B0
:10039000948CE994005005755B00811D882178A23A
:1003A000E6A8216055C3E894C8E994005008E4D257
:1003B000E4FB7A0A61F8C3E89468E994015008E420
:1003C000D2E3FB7A0F61F8C3E894D0E994025008B5
:1003D000E4D2E2FB7A1E61F8C3E894A0E9940550E8
:1003E00008E4D2E1FB7A3C61F8C3E89498E9940808
:1003F0005008E4D2E0FB7A787E00C3E89559FCE926
:10040000955AFD30E70AECF42401FCEDF43400FDCC
:10041000755B00C3EC9AED9E5003755B01885989AA
:100420005A8557558558567802A153C3E89527F841
:10043000E99528F9307C02A137307B02A137307A68
:1004400002A130207502814EE9FDE8FC816DE9C30F
:1004500013F9E813F8307902A130E9C313F9E8136E
:10046000F8307802A130E9C313FDE813FC20612CB9
:0F047000C3EC941CED940240028184ED701EC316
:10047F00EC94C850180529E52970021529C3E52900
:10048F00940A5002A16B755C00D270A16BE52960D4
:10049F000215297888E6F97400207F087896B90349
:1004AF0002789EE624FAFEE43400FFC3EC9EFCEDD6
:1004BF009FFD9208B90310A2085007207609D27643
:1004CF0081D6307602C276A2085016B9030DECF42D
:1004DF002401FCEDF43400FD0204F078007900A152
:1004EF0037B90315EC33FCED33FDC3EC940AFCED87
:1004FF009400FD50047C007D00C3EC94FFED94004C
:10050F00400678FF7900A137EC8572F0A4C5F0A200
:10051F00F733F87900400302055378FF790002059D
:10052F0053E9C313F9E813F8307C0EE9600278FF42
:10053F00C3E81338F8E43400F9C3E894FFE99400F2
:10054F00400278FF885CD270206102A16B741FF4A7
:10055F00552F4BF52FC274EB7002D274752A1830D9
:10056F007403752A0A306102A17F20740353DAFEE7
:10057F00207403752B06D0F0D0E0D0D0D2AD43E677
:10058F00103279010205AF79030205AF790A02052E
:10059F00AF791E0205AF79640205AF79C80205AFC6
:1005AF007817E4D5E0FDD8FAD9F6227A147B7802D1
:1005BF0005D67A107B8C0205D67A0D7BB40205D650
:1005CF007A0B7BC80205D67902E4D291D5E0FDD231
:1005DF0094D5E0FDC294D5E0FDC291D5E0FDE920B0
:1005EF00E002D29530E002D293E573D5E0FDE92029
:1005FF00E002C29530E002C2937496D5E0FDD9C9EE
:10060F00EAF8D5E0FDD8FBDBBED29122C37C007D9A
:10061F000075F00005F0EA33FAEB33FB50F6EB13FD
:10062F00FBEA13FAC3E9FFE8FEE89AF8E99BF950F1
:10063F0004EFF9EEF8B3EC33FCED33FDD5F0DFED5D
:10064F00F9ECF822E889F08A20D2D4F8A9F07B00DF
:10065F0030F70B7BFFF42401F8E9F43400F9E88557
:10066F0020F0A4ADF0F8E98520F0A4AFF0FEED2E58
:10067F00F974003FFA7C04C3EA13FAE913F9E8139B
:10068F00F8DCF48BF030F70AE8F42401F8E9F434DD
:10069F0000F9E889F0C2D4F8A9F0227882B60403F1
:1006AF00020705C3E55C940140030206CF852224AF
:1006BF00E4F544F545F546F547F548C26E020705E2
:1006CF007882E6FCD26EE522F523783879C7AA4006
:1006DF00AB41C3EB13FBEA13FAEC146013C3EB1338
:1006EF00FBEA13FAEC14146007C3EB13FBEA13FADB
:1006FF00D11B8844894522C3E5449523F8E54594E9
:10070F0000F9500CC3E89480E994FF4016020736B5
:10071F00C3E8947FE994005003020736787F79008D
:10072F00020736788079FF8849894A22E5492546AC
:10073F00F8E54A3547F9854A20E4300701F4354892
:10074F00FA30E709C3EA94F04015020774C3EA943C
:10075F000F500302077478FF79FF7A0F020774783E
:10076F000079007AF0C3E5249561500AC3740195AE
:10077F0024500B020792E54A20E70E020792E54A42
:10078F0030E706884689478A482278A5E6FAC3E506
:10079F004933F8E54A33F9D153E930E70BC3E8940D
:1007AF0080E994FF4013E1CCC3E8947FE9940050B3
:1007BF0002E1CC787F7900E1CC788079FFE820E7FF
:1007CF0015C3E52398F84009C3E8940140030207D5
:1007DF00F378010207F3E8F424012523F84003021C
:1007EF0007F378FF884B2278A6E6FAA847A94812A4
:1007FF000653E930E70CC3E89401E994FF40160271
:10080F000828C3E894FFE99400500302082878FFF2
:10081F007900020828780179FFE920E715C3E54B35
:10082F0098F84009C3E89401400302084F78010289
:10083F00084FE8F42401254BF8400302084F78FFD6
:10084F0088242278FFC26420693D206A12D264C3D3
:10085F00E541940A4009C3E52594405002C26479EA
:0E086F00A1E76023E541601F74FF8541F0841E
:10087D008539F0306A0375F005A4F8C5F06002788B
:10088D00FFC3E895645002A864886322C3E54094D1
:10089D0040E5419401E56350031401AA046002F59B
:1008AD0063220208B22275E890227883E6FFE5E81C
:1008BD0020ECF7A8BDA9BE0570C3E57094084052A1
:1008CD00757000E9FA79A0E76044EA7007E5716098
:1008DD001B0208EDC3E895716010E5715006600CC0
:1008ED00140208F90460F90208F9E571F571C39471
:1008FD006D401B7561C0C394044013756180C39432
:10090D0004400B756140C39404400375610075BBD1
:10091D000622E5612410500274FFF5617982B70457
:10092D00022146C3A861E524985002A824C3E89586
:10093D00634002A86388258826E570B4070375BB5C
:10094D001022743279A787F0A4C5F0A2F733F8C34B
:10095D00E895614002A86188228824882588268828
:10096D0064227540007541F022C2AF75C820A8CC35
:10097D00A9CDAA3A30CF010A75C824D2AFAB3BAC92
:10098D003C883B893CC3E89BF8E99C206908F93019
:10099D006702418221DFAD3D8A3DF9EA9DFA60048F
:1009AD0078FF79FFAE3EAF3F8B3E8C3FA83BA93C15
:1009BD00C3E89EF8E99FF9C3E54113FBE54013FA3F
:1009CD00E82AF540E93BF54150067540FF7541FFBA
:1009DD004129AA40AB41AC40AD417E047F02C3EB3F
:1009ED00940440021E1FC3EB940840021E1FC3ED6A
:1009FD0013FDEC13FCDEF7C3EA9CFAEB9DFBEF60F5
:100A0D0009C3E913F9E813F8DFF7EA28FAEB39FB24
:100A1D008A408B4150067BFF8B408B41C3EB940288
:100A2D005002D2673069047F0341547892E6FFC3C8
:100A3D00E537948240110FC3E53794A040010FC3F1
:100A4D00EF940640027F057E02E541C4540FF9E59F
:100A5D0041C454F0F8E540C4540F28F8C3E89EFA99
:100A6D00E99400FB4009C3EA9402EB940050047A28
:100A7D0002E4FB41CEAA40AB41EBC4FEEAC4540FE5
:100A8D004EFCC3EA9CFAEB9400FBC3E813C313F8C6
:100A9D00EA28FAEB3400FB8A408B41C3EB94024009
:100AAD0002C2677802EBC4FE7B00EAC4540F4EFA13
:100ABD00C3EA98FA4005C3940250027A027892E68E
:100ACD00FF30600241CE855192855293D26043E64C
:100ADD0080C3E49AF8E49BF9306702615AE8FAE9B9
:100AED00FBD3E913FDE813FC88518952C3EF94033E
:100AFD006038EF20E00DE82CF8E93DF9ECFAEDFB5C
:100B0D00020B23E828F8E939F9C3E82402F8E9349F
:100B1D0000F97AFE7BFFC3EF9403400E8A538B548A
:100B2D00884D894E8C4F8D50618E885389548A4DD6
:100B3D008B4E8C4F8D503069127553F07554FF7577
:100B4D004FF07550FF7551F07552FF618EE8FAD375
:100B5D00E813FC8851C3EF94036020EF20E007E811
:100B6D002CF8ECFA617AE8282402F87AFEC3EF94A7
:100B7D000340088A53884D8C4F618E88538A4D8C63
:100B8D004FE568C3335002646BF5683060026198BD
:100B9D00753402D26043E680E52D54066034A840DA
:100BAD00A941C3E913F9E813F8C3E913F9E813F8F8
:100BBD00306904E92440F9C2AF53E67F759100C353
:100BCD00E498F594E499F595759104D26043E68027
:100BDD00D2AF22D265754300752000306C037520AD
:100BED0040020BFFD265754300752040306C0375D4
:100BFD00200078017901206720E52D54066002C29E
:100C0D00657914E541C313700104F8C394144002CF
:100C1D007814306904781B791B206010E543600C53
:100C2D00306903D53404D26D81A171A00543E59BD4
:100C3D005440B52002818B30690908C3E899400101
:100C4D0018812620650A08C3E899400261FF8126B4
:100C5D00C265C2AF53E67F7591003067127594007F
:0F0C6D007595FE759104D26043E680D2AF61FFAA
:100C7C00AE40AF41C3E49EF594E49FF5958170C3FB
:100C8C00E5339401500261FF30650261FFD80281A7
:100C9C009F8126C26DC2AF53E67F75910085539438
:100CAC00855495759104854D92854E93D26043E69B
:100CBC0080D2AFE52D54066008206A020533020C81
:100CCC00DD306D0D206C0A2065071581158102152C
:100CDC00682278003064053065027801E53775F0DC
:100CEC0007A4F9E5F028F5F0E9A2F013A2F113A29C
:100CFC00F213F537C394785003753778C3E53795FD
:100D0C00384008D266C295C294C293306002A117D3
:100D1C00854F92855093D26043E68022207D16C287
:100D2C00AF754202D291C292306202D293D2AF75A9
:100D3C009F11020F1FC2AF754202D291C290306256
:100D4C0002D295D2AF759F11020F1F307245207DD4
:100D5C0022C2AF754203900135757B02C293D290CB
:100D6C00D292306204D294A177C291D2AF759F0116
:100D7C00020F1FC2AF754203900135757B02C295FD
:100D8C00D292306204D294A197C291D2AF759F21B6
:100D9C00020F1F207D17C2AF754203900110C29342
:100DAC00306202D294D2AF759F01020F1FC2AF7591
:100DBC004203900110C295306202D294D2AF759F5B
:100DCC0021020F1F207D16C2AF754204D292C29031
:100DDC00306202D294D2AF759F21020F1FC2AF7541
:100DEC004204D290D292C292306202D294D2AF75A7
:100DFC009F01020F1F307243207D20C2AF75420548
:100E0C00900124757B04C294D291306204D295C1B6
:100E1C001FC292D2AF759F11020F1FC2AF75420550
:100E2C00900146757B01C294D291306204D293C179
:100E3C003FC290D2AF759F11020F1F207D17C2AF1A
:100E4C00754205900106C294306202D295D2AF75FC
:100E5C009F11020F1FC2AF75420590011AC2943048
:100E6C0062EBD293D2AF759F11020F1F207D18C277
:100E7C00AF754206D290D292C291306202D295D214
:100E8C00AF759F01020F1FC2AF754206D292C2917D
:100E9C00306202D293D2AF759F21020F1F30724580
:100EAC00207D20C2AF754201900146757B01C29531
:100EBC00D292306204D293C1C7C290D2AF759F2137
:100ECC00020F1FC2AF754201900124757B04C293BF
:100EDC00D290D292306204D295C1E9C292D2AF754F
:100EEC009F01020F1F207D17C2AF75420190011A9E
:100EFC00C295306202D293D2AF759F21020F1FC2EE
:100F0C00AF754201900106C293306202D295D2AF06
:100F1C00759F01C26622900104757B00C295C29434
:100F2C00C293D292D291D290C26222788076090872
:100F3C0076090876040876FF0876030876FF0876AB
:100F4C000A087601087601087601788C7601087615
:100F5C00FF0876FF0876FF0876FF0876FF08760311
:100F6C000876FF0876FF0876FF0876250876D00805
:100F7C0076280876500876040876FF0876020876FC
:100F8C000008767A0876FF08760108760108760064
:100F9C00087603087600227887E6FFC2727888E626
:100FAC00C394036008C27DE630E102D27DC27E7834
:100FBC0089E630E102D27EC3EF94026008758E019F
:100FCC00D273020FD6758E00C273227880E614900D
:100FDC0000809378A5F67881E6149000809378A62B
:100FEC00F67886E61490008D9378A7F67886E6F569
:100FFC0039C394025003753902789CE67538FFB4F6
:10100C0002037538A0B4030375388278A3E61490F4
:10101C00009A93F566120F2222227896E6FA7897B8
:10102C00E6FB7888E6B40305C3EB940EFB307F0433
:10103C007A007BFFC3EB9AFCC3948250027C8275CE
:10104C0072000572EC8572F0A4C3E5F0947D40F259
:10105C0022D27F11261205A07A007B007C1012058B
:0F106C0096E55C2AFA74003BFBDCF37C04C3EBD3
:10107B0013FBEA13FADCF7FEC27F112622E5EF2001
:10108B00E6037520000520903FFFE52014600690D5
:10109B001DFF1460009304600375EF1253D9BF75E5
:1010AB0081C043FF8012059175EF0243B203E5B394
:1010BB00240220E70DF521E5E320E0068521B3436B
:1010CB00E301120F227580FF75A40075F19075D4A2
:1010DB007F75908775A5BF75F2BF75D50075A60195
:1010EB0075E241120F22E4F8F6D8FD756801120F74
:1010FB00371215B978988673753001C2AF1205AAED
:10110B001205BA1205A01205C11205A01205C812CC
:10111B0005A0C2AF78FA79FA308707D9FBD8F70266
:10112B001C00120FA3120FD7112511267898867366
:10113B00120F2275881075890275C8247591047574
:10114B00D84075A82275B80275E690759B80759D81
:10115B000075D10E75BC5875BB0675BA1175E88054
:10116B00120591D2AF1208AF75360053DACF207E3D
:10117B000343DA20307E0343DA1043DA01C2D8C2CC
:10118B00711205AAD2617B037A0CE55B70077A0CAE
:10119B00DB0302111D1205A020700302111DC2708A
:1011AB00E55CC3940240E1E52F541F855E5DF55E5F
:1011BB00B55DD5DAD5C26153DACF207E0343DA2091
:1011CB00307E0343DA10C2D8C27178A2E67008D21F
:1011DB0074E52F54E0F52FC2757529001205A53063
:1011EB007409C3E529940A4002D275120596780258
:1011FB003074027800C3E55C9840F0C2AF1205BAB8
:10120B001205BA1205BAD2AF1205AA754C0078882E
:10121B00E6B4030241F5120596788CE6C3940150AF
:10122B00030212F5E530C3940150030212F520744A
:10123B0035C3E55C94FF50030212F5C2AF1205CF24
:10124B00D2AF1205A5C3E55C940150EFC2AF1205F6
:10125B00BA12059B1205BAD2AF1205A5C3E55C9471
:10126B00FF40E90217617F02D27F11261205A5C24A
:10127B00AFC27F1126AE5CC3E55C947FD2AF4074E6
:10128B00120591C2AF1205CFD2AFDFDC115DC3EEF9
:10129B007897F61205AA1215FB1216E47F0AD27F75
:1012AB0011261205A5C2AFC27F1126AE5CC3E55C49
:1012BB00947FD2AF50E6120591C2AF1205BA120558
:1012CB009B1205BAD2AFDFD6115DEE24037896F6EA
:1012DB001205AA1215FB1217131205A51126C3E549
:1012EB005C94FF50024139021761C3E55C954C4099
:1012FB0003855C4C1205A578017988E7B403027865
:10130B0005C3E55C9840024119C2AF1205CF120527
:10131B00CF1205CFD2AF1205AA753000E4F531F527
:10132B00320531E531F4703F0532789AE6781914BD
:10133B006012783214600D787D14600878FA1460AE
:10134B0003753200C3E53298401D120F221205912E
:10135B00153275310078998673C2AF1205CFD2AFB3
:10136B00789886731205A512059BE52A70053074D3
:10137B0002211D78012074027806C3E55C9840A118
:10138B007888E6C3940360031205A5E52A7003026F
:10139B00111DC2AF120F22E4F522F523F524F5251A
:1013AB00F526F567D2AF7885E6C333F565E4F544EA
:1013BB00F545F546F547F548F570F52CF52DF53760
:1013CB0075700875BB101205911208B3E5E820EC97
:1013DB00FBA8BDA9BEE97001F888711208B775703A
:1013EB000875BB10120FA3C2AF7561FF12094F85B1
:1013FB002261852262852263D2AF75220175240199
:10140B00752501752601856069756A017888E6B4D2
:10141B000307C27D307602D27DD268D26975330064
:10142B00120E78120EA912096F12097612096F1299
:10143B00097612096F120BF11206AA120CDE120DAD
:10144B0028120976120BE0306E0312070620670391
:10145B00120852306703120899120CDE120D571244
:0E146B000976120BF1306E0312073B120CDEF5
:10147900120DD0120976120BE0306E031207991281
:101489000CDE120E01120976120BF1306E031207EF
:10149900F6120CDE120E781209761208B3120BE05E
:1014A900120CDE120EA91208B712097630693285BC
:1014B9006461856462856069756A0179187A0CC30B
:1014C900E53399400FC269D26A8A358564618564BA
:1014D900630214EAC3E55C94014003021440021557
:1014E90070306A1D206C1AE535147006C26AD26B19
:1014F9008140F535C3E55C940140030214400215AF
:101509007075360078FA79A4E760027803C3E55F5D
:10151900985054307404E52A604D7888E6B403176E
:10152900207D05207607A140307602A140206C0776
:10153900D26C856461817F78F0306C05856461784F
:1015490020C3E5419850028140306C1BC26CC27DBA
:10155900307602D27DD26A75351285646181400583
:1015690036E55C6002A173753600C2AF120F2278AE
:1015790087E6FE7602120FA37887EEF6E4F522F5E8
:1015890023F524F525F526F565752C00752D00D272
:10159900AF1205A5120F2278A4E66006C292C29185
:1015A900C290307409C3E53694044002211D6127B5
:1015B900901A0D782012163DE520B4550CA3121689
:1015C9003DE520B4AA030215DB120F371215FB0201
:1015D90015FA901A0378807B0A12163DA308DBF9E5
:1015E900901A0F788C7B1912163DA308DBF9901A13
:1015F9002822C2AF12167C121656901A00740E12C7
:101609001642A37406121642A37415121642901AB2
:101619000378807B0A121641A308DBF9901A0F7828
:101629008C7B19121641A308DBF912168F12166D5D
:10163900901A2822E493F622E6438F01538FFD7511
:10164900EF0275B7A575B7F1F0538FFE22438F02EC
:10165900438F0175EF0275B7A575B7F1901A0DF0B3
:10166900538FFC22901A0D7455D142901A0E74AA08
:10167900D142227A3079D07820901A40D13DE520A4
:10168900F709A3DAF7227A3079D0901A40E7D142E4
:1016990009A3DAF922AB74A875BB01027980BB02F0
:1016A900027981BB03027982BB04027984BB0502FA
:1016B9007986BB06027992BB07027987BB08027952
:1016C900A3BB0902799CBB0A027988BB0B02798901
:1016D900E8F7227C051205AADCFB22C2AF1205BA83
:1016E9001205C11205C81205CF12059B1205BA12BF
:1016F90005C11205C81205CF12059B1205BA1205BC
:10170900C11205C81205CFD2AF22C2AF1205CF123E
:1017190005C81205C11205BA12059B1205CF12059B
:10172900C81205C11205BA12059B1205CF1205C8C8
:101739001205C11205BAD2AF22AE74AF75C2AF128B
:1017490005BA1205BA1205BA12059BDEF21205CFC7
:1017590012059BDFF8D2AF22D1E4D1DCD1DC75745C
:1017690001757501757600F1427C05AD5C1205AA1B
:10177900C3ED955C70F5C3E55C9401400AC3E55C73
:1017890094FF403202179DD19EB1FBD1E4C2AF75DF
:10179900EF12D1DCDCD50576C3E5769403500280DF
:1017A900C6D1DC0575E5741490009F93F808C3E56C
:1017B9007598500280AED1DCD1DC0574C3E5749410
:1017C9000C5002809C120F37B1FBC2AF75EF12D1DA
:0117D900DC33
:0319FD000210884D
:101A00000E0615090904FF03FF0A01010155AA0189
:101A1000FFFFFFFFFF03FFFFFF25D0285004FF0259
:091A2000007AFF0101000300FF40
:101A400023585032354123202020202020202020E0
:101A500023424C48454C4923463333302320202031
:101A60002020202020202020202020202020202076
:101C0000C2AFC2D353D9BF7581C043B20343FF8073
:101C1000752438752503B1C975EF0275E24043F1AB
:101C20008053A47F75D4FFD2877DFA780379E67C50
:101C300010752200752300901DD67B0675249875BB
:101C400025013087028142208708D8FBD9F9DCF7CB
:101C500081B4308708D8FBD9F9DCF781B4B189E4C5
:101C600093A3C39A6004DDC381B4DBDBB17B600264
:101C7000812B7B08E493FAA3B15CDBF87A30B15C8A
:101C8000752200752300B17BEAFCEBFDC3ED94FEE9
:101C9000400EB17B8A278B28ED30E0048A828B834B
:101CA000B17B7AC270D8C3ED94FE601350CEBD00F4
:101CB00025EC60097520007521FF0200008100A855
:101CC00027A9280809D804D90281D3B17FEA89AAB3
:101CD000F281C50D81A0C3ED94035049EDA2E092BD
:101CE000007AC5C3E5829400E583941C50902000DF
:101CF00010438F02438F0175B7A575B7F1F030001F
:101D00001FA827A9280809438F01538FFDD804D99C
:101D100002A12089AAE275B7A575B7F1F0A3A10DBC
:101D2000538FFC817C7AC1BD030CE493A3FAB140CC
:101D3000DCF8B138817C817EAA22AB23B15CEBFA5E
:101D4000EA6222752608C3E52313F523E52213F57D
:101D50002250066323A0632201D526EAB1C9B1C986
:101D600075260AEAF4200102D287300102C287B147
:101D7000C9C3134002C201D526EB22B17FEAFB2082
:101D80008702A17F308702A184752608AE24AF2583
:101D9000C3EF13FFEE13FEB1CDB1C9C3EA13308711
:101DA000024480FA30E703632201C3E52313F523DD
:101DB000E52213F52250066323A0632201D526D91C
:101DC000E52265236523F52222AE24AF250E0FDE22
:101DD000FEDFFCD20122424C48656C693437316326
:041DE000F3300601D5
:00000001FF
